:100000008013002051140000774900003D140000C7
:100010003D1400003D1400003D14000000000000ED
:10002000000000000000000000000000911200002D
:100030003D140000000000003D1200003D140000CF
:10004000F5110000F5110000F5110000F511000098
:10005000F5110000F5110000F5110000F511000088
:10006000F5110000F5110000F5110000F511000078
:10007000F5110000F5110000F5110000F511000068
:10008000F5110000F5110000F5110000F511000058
:10009000F5110000F5110000F5110000F511000048
:1000A000F5110000F5110000F5110000F511000038
:1000B000F5110000F5110000F5110000F511000028
:1000C000F5110000F5110000F5110000F511000018
:1000D000F5110000F5110000F5110000F511000008
:1000E000F5110000F5110000F5110000F5110000F8
:1000F000F5110000F5110000F5110000F5110000E8
:1001000053B94AB9002908BF00281CBF4FF0FF317E
:100110004FF0FF3000F06CB9ADF1080C6DE904CE82
:1001200000F006F8DDF804E0DDE9022304B07047D2
:100130002DE9F047089E0D4604468E46002B40F000
:1001400082808A42174646D9B2FA82F24AB1C2F197
:10015000200105FA02F320FA01F1974041EA030E6B
:1001600094404FEA1748230CBEFBF8FCB9B208FBD9
:100170001CEE43EA0E430CFB01F098420AD9FB182F
:100180000CF1FF3580F01681984240F21381ACF1FA
:10019000020C3B441B1AA4B2B3FBF8F008FB10336B
:1001A00044EA034400FB01F1A14209D93C1900F1E2
:1001B000FF3380F00181A14240F2FE8002383C44CE
:1001C000641A40EA0C4000211EB1D4400023C6E965
:1001D0000043BDE8F08702B9FFDEB2FA82F2002ADE
:1001E0004FD1CB1B4FEA174E1FFA87F80121B3FB03
:1001F000FEFC250C0EFB1C3345EA034508FB0CF303
:10020000AB4207D97D190CF1FF3002D2AB4200F2AC
:10021000E7808446ED1AA3B2B5FBFEF00EFB105545
:1002200043EA054408FB00F8A04507D93C1900F152
:10023000FF3302D2A04500F2D7801846A4EB080491
:1002400040EA0C40C0E78B4208D9002E00F0AF8096
:100250000021C6E900050846BDE8F087B3FA83F13E
:1002600000294BD1AB4202D3824200F2B780841AFC
:1002700065EB030301209E46002EAAD0C6E9004E7E
:10028000A7E7C2F1200C01FA02F3974020FA0CF024
:100290004FEA174E21FA0CFC1843BCFBFEF1050C8B
:1002A0000EFB11CC1FFA87F845EA0C4501FB08F359
:1002B000AB4204FA02F409D97D1901F1FF3C80F048
:1002C0008B80AB4240F2888002393D44EB1A85B204
:1002D000B3FBFEF00EFB103345EA034500FB08F3C9
:1002E000AB4207D97D1900F1FF3C71D2AB426FD907
:1002F00002383D44EB1A40EA014178E7C1F1200C95
:100300008B4022FA0CF71F4320FA0CF405FA01F394
:100310004FEA174E25FA0CF51C43230CB5FBFEF9EA
:100320001FFA87F80EFB195543EA054509FB08FA41
:10033000AA4502FA01F200FA01F308D97D1909F180
:10034000FF3047D2AA4545D9A9F102093D44A5EBA2
:100350000A05A4B2B5FBFEF00EFB105544EA0544B5
:1003600000FB08F8A04507D93C1900F1FF352DD254
:10037000A0452BD902383C4440EA0940A4EB0804CC
:10038000A0FB02894C45C6464D4619D316D05EB136
:10039000B3EB0E0264EB050404FA0CFCCA404CEA11
:1003A0000202CC40C6E900240021BDE8F0873146B6
:1003B00030460EE7AC46EDE6184601E74345E6D287
:1003C000B8EB020E69EB07050138E0E72846D3E7F2
:1003D00060468FE78146BAE7614677E708464BE714
:1003E000ACF1020C3D4415E702383C4426E700BF5F
:1003F000704700BF70B5164802F0B2FF044630B334
:1004000002698168136843F4005313600B6840F27B
:1004100001620D219847002819DB012523691B681B
:1004200085F0010613F4005F18BFF5B265B1A3684B
:10043000DB684FF4005120469847F5B200214FF495
:10044000004003F091FCE9E7A3681B69F1E770BD88
:100450004C5500002DE9F04F91B08B46029092462A
:100460001C4600259AF8000008B928465EE32528B6
:100470000AF1010707D0029B594698470028C0F2AD
:100480005583013510E2182200210AA804F0AEFAC3
:100490009AF80130252B78D00022944616469646CD
:1004A0001046394617F8013B2B2B00F09D8000F2D7
:1004B0009480202B00F09B80232B00F09A8028B1A1
:1004C0009DF8300040F004008DF83000BEF1000FC0
:1004D00005D09DF8300040F008008DF830002EB1B6
:1004E0009DF8300040F010008DF83000BCF1000F96
:1004F00005D09DF8300040F020008DF830002AB182
:100500009DF8302042F040028DF830209DF83020D8
:1005100002F04400442803D16FF386128DF8302096
:100520009DF830202A2B42F080028DF830207BD1BC
:100530009DF8312042F001024B1C8DF831201A78D1
:100540002E2A9DF831200CBF0121002161F34102C8
:100550008DF8312074D15A782A2A6AD001330021CB
:100560000A26184610F8012BA2F13007092F40F295
:100570008E809DF830200E91C2F3400040EAD17188
:1005800061F341028DF830205AE00AF102078DF83C
:1005900033309DF83130D90740F1498154F8049B3C
:1005A000B9F1000F07DA9DF8302042F004028DF80F
:1005B0003020C9F100095A0740F1428154F8048BF8
:1005C000B8F1000F80F241819DF831306FF34103A3
:1005D0008DF831304FF0FF3837E12D2B0CD0302B18
:1005E0007FF46DAF01225CE74FF0010E59E7012661
:1005F00057E74FF0010C54E7012052E70CFB0202D1
:10060000303A33461E4616F8010BA0F13007092F89
:10061000F4D9994293D09DF830100D92D20F62F325
:1006200041018DF830108AE70B4600224FF00A0C8A
:10063000E8E79DF8312042F004028DF831200233C2
:100640001F4617F8012B6C2A41D025D8682A2BD0D9
:100650006A2A46D04C2A4CD01F4617F8012B9DF829
:1006600031308DF83320782A00F2D980572A4DD8BE
:10067000412A03D0453A022A00F2D1809DF8323057
:10068000042262F302038DF8323001239EE006FB60
:1006900001213039034664E7742A26D07A2ADBD157
:1006A0009DF8313006220DE05A78682A9DF83120F5
:1006B00006D1012161F3C6028DF831209F1CCCE7E1
:1006C0001346022262F3C6038DF83130C5E75A782B
:1006D0006C2A9DF8312001D10421EBE71346032257
:1006E000F0E79DF831300522ECE79DF83130072224
:1006F000E8E7BDF8303023F4F04323F0020343F47D
:10070000804343F00203ADF83030A6E7A2F1580170
:10071000202900F2848001A050F821F0E1070000B8
:100720001F0800001F0800001F0800001F0800002D
:100730001F0800001F0800001F0800001F0800001D
:100740007D0600001F080000E1070000A10700006F
:100750007D0600007D0600007D0600001F080000E9
:10076000A10700001F0800001F0800001F0800006C
:100770001F080000E9070000E1070000050800006D
:100780001F0800001F080000050800001F080000E7
:10079000E10700001F0800001F080000E10700003B
:1007A0009DF83210012003F0780360F30201402B22
:1007B0008DF8321002BF9DF8301041F001018DF824
:1007C0003010632A31D1003B18BF01239DF830203F
:1007D000C2F340010B4363F341028DF83020D8E6A9
:1007E0009DF832100220DEE79DF8322003F07803F6
:1007F000A3F14000032161F3020243428DF832204D
:100800004341E3E79DF83220032113F0780F61F3B1
:1008100002028DF8322014BF01230023D6E79DF891
:10082000303043F001038DF830300023CEE79DF9DE
:100830003020002AB4BFDDF834904FF0FF39BAE61B
:100840009B077FF5C7AEDDF838809DF83120002387
:10085000CDE90D339DF8323003F00703012BC2F3CD
:10086000C30236D1D31E042B20D8DFE803F00307E0
:10087000071F1F0054F8040BC11704E0073424F0CD
:100880000704F4E80201CDE90A019DF8303013F0C5
:10089000030654D002983B465246594603F05FFF88
:1008A0000028C0F243810544BA46DBE554F8040B46
:1008B000012A4FEAE071CDE90A0105D19DF82830FF
:1008C0000A9300230B93E0E7022ADED1BDF928004A
:1008D000D2E7022B23D1D31E042B13D8DFE803F079
:1008E000030A0A12120020680A900021231D0B91AE
:1008F0001C46CAE7073424F00703F3E80201CDE9F8
:100900000A01F5E754F8043B0A93012A4FF000036B
:100910000B93D3D0022AB8D1BDF82830D0E7042BEE
:1009200007D1073424F00704F4E80201CDE90A01F5
:10093000ABE7032B04BF54F8043B0A93A5E79DF8EB
:1009400033007828B0D8622822D825283FF493AD08
:100950005828A9D10DF126030093DDE90A0104AB63
:100960000CAA03F0B1FE8246B8F1000F0DF126008B
:100970000CDB9DF83020A0EB0A036FF3861298453C
:100980008DF8302002D9A8EB03030D9380463DE09B
:100990006338152888D801A151F820F01D0A0000FD
:1009A000810A0000A9080000A9080000A9080000A9
:1009B000A9080000810A0000A9080000A908000099
:1009C000A9080000A9080000DF0A0000AD0A000025
:1009D000B10A0000A9080000A9080000F5090000FC
:1009E000A9080000AD0A0000A9080000A90800003D
:1009F000AD0A0000B8F1000FDDF828A00ADB41467F
:100A0000504603F0D3FF0AEB00080026BAF1000FAE
:100A10000CD149E7504603F0C2FFF4E70A9B8DF87A
:100A2000103000260DF111080DF1100AA8EB0A0391
:100A300006B101339DF83220D0066BD50233520641
:100A40000D9948BF0E9A0B4448BF9B18B9F1000F8F
:100A500079DD9DF83020A9EB0309C2F380030393ED
:100A6000530770D4500664D546B1029B59463046B0
:100A7000984700285ADB039B01351E46302359E076
:100A80001E0711D413F0100618BF2026DDE90A2333
:100A9000002A73F10001BFF65DAF524263EB4303DE
:100AA000CDE90A232D2655E72B26EFE7002651E74F
:100AB0000A9848B30DF1260300930CAA04AB002159
:100AC00003F002FEBDF8323003F0EF0343F4F043CD
:100AD00043F010038246ADF83230002644E70A9B0B
:100AE000072A3FF6E1AEDFE802F00D04060D080824
:100AF0000D0D1D70D8E61D80D6E62846E917C3E91E
:100B00000001D1E61D60CFE6DFF8C4800646A8F1FB
:100B1000050A8BE7110748BF013390E71846039396
:100B20005946029B98470028039B04DA11B0BDE8A0
:100B3000F08F20234D444A46002AA5EB090109F114
:100B4000FF39EBDC0D4636B1029B594630469847DB
:100B50000028EBDB01359DF83230D90601D41A07A5
:100B600006D5029B5946302098470028DEDB013528
:100B70009DF83230DB0607D59DF83300029B5946BD
:100B800098470028D2DB01350D9E2E44731B002BA5
:100B900016DC029843465246594603F0E0FD002811
:100BA000C4DB0544A944A9EB0503002B7FF77CAE09
:100BB000029B5946202098470028B7DB0135F2E711
:100BC000029B5946302098470028AFDB0135DDE70E
:100BD00058550000014803F0E5BB00BF88530000F2
:100BE00008B5D0B14368042B11D100220368BFF3CC
:100BF0005B8F53E8001F012903D143E80020002840
:100C0000F7D1BFF35B8F074808BF104608BD3BB163
:100C1000006802F079FD0020F8E76FF4E040F5E7A6
:100C20000148F3E7E98FFFFFEA8FFFFF10B50446A5
:100C300018B90D4B0D485B689847616808290DD0BD
:100C400031F004030AD011F0020108D0084821460F
:100C500004F025F9002323600023636010BD2068A1
:100C6000142203F0C3FEF7E7DC0000205955000012
:100C7000C802002010B5044618B9164B16485B6828
:100C800098476368042B23D0082B21D0CBB9236865
:100C9000BBB912484FF0FF324FF0FF33214602F04C
:100CA00085FC08B923681BB90A4B0D485B68984757
:100CB00020681422002103F099FE636843F00203C8
:100CC0006360206804F014F9636843F00103636013
:100CD00010BD00BFDC00002059550000C8020020F4
:100CE0007F55000008B508B34368042B10D10122DA
:100CF0000368BFF35B8F53E8001F002903D143E86B
:100D000000200028F7D1BFF35B8F0BD1002008BD76
:100D100053B100684FF0FF324FF0FF3302F076FC22
:100D20000028F3D00348F2E70348F0E76FF4E0400F
:100D3000EDE700BFE98FFFFFEA8FFFFF08B5064927
:100D400006484023142204F08FF8BDE80840044907
:100D5000044803F089BB00BFE4020020C802002061
:100D6000A0530000905300002DE9F84FB0F8189000
:100D700019F00808044693460DD001290CBF49F02C
:100D8000100949F02009A0F818908BF31188BFF3DF
:100D90006F8FBDE8F88F09F00709022907D12046B7
:100DA00003F016FD0028F0D00128238B50D167698D
:100DB000218B002F15DA256821F00701C4E900888E
:100DC00041F0010121830026218B01F0070ACA4569
:100DD00002D0A368002B5CD10DB9002E74D0002383
:100DE00058E001F007035A1F012A20D821F007011B
:100DF000062B256889B2C4E900880CD1002D2B464A
:100E000038BF00232BB1628B1B6801326283002B39
:100E1000F8D141F002012183204603F0D9FC0646B7
:100E20000028D1D0238B43F020032383CBE7042B6E
:100E30000CD121F0070189B22183204603F0C8FCC0
:100E400005460028BFD041F0200121830025BAE7E4
:100E5000032809D1226923F00703166843F006032B
:100E6000238300252F46AFE7042806D1226923F00B
:100E70000703566843F00403F2E7052806D1226908
:100E800023F00703966843F00503E9E700252E46A3
:100E9000E8E7012341F0080121838BF31188BFF3B8
:100EA0006F8F03BB002D33D116B121492046B047C7
:100EB0004FF02003EFF3118B83F31288BFF36F8F92
:100EC000238B23F008032383238BDA0628D523F012
:100ED000100323830121B4F8189009F007090029B1
:100EE0007FF45BAF51E7A1680029DBD00B68D1F834
:100EF00004B0002B38BF0023994652463B4620469B
:100F0000D847B9F1000FCDD0D9F800304946EEE707
:100F100029463B46524620462D6803F075FCC1E742
:100F200013F020011EBF23F0200323830221D2E708
:100F3000354800002DE9F84305464FF02003EFF354
:100F4000118683F31288BFF36F8F104B1C68002C3F
:100F500038BF00249CB10E4FDFF838804FF00C09E9
:100F6000D4E90132002D08BF13462BB198F81420A4
:100F700009FB02F2B85C98472468002CF0D186F394
:100F80001188BFF36F8FBDE8F88300BFE40700202E
:100F9000F00700204C09002000F01F0301229A40B6
:100FA0000A4BBFF35B8F400903EB800050E8003F22
:100FB00043EA020140E8001CBCF1000FF6D1BFF388
:100FC0005B8F1A4214BF012000207047FC070020ED
:100FD00030B51D4B1D7DBFF35B8F05F01F03012254
:100FE0009A401A4B690985B0D04303EB810353E85B
:100FF000001F01EA000443E8004CBCF1000FF6D1E9
:10100000BFF35B8F114217D0114C0C2202FB05423B
:1010100007CA01AB83E807000E4A7AB193E80700DC
:1010200003F000FD0020FFF785FF0C236B43002237
:10103000E118E250C1E9012205B030BD82F3118808
:10104000BFF36F8FEEE700BF4C090020EC070020D4
:10105000F0070020254A00002DE9F041374BDFF86A
:10106000F4801C7D88B007462046FFF795FF60B9E5
:101070006E463A462146304603F064FC96E8070087
:101080000C2505FB048585E807000C23634308EB6A
:10109000030218F80300650904F01F06C8B37B1C9F
:1010A0000FD0D2F808E02648264A4FF4004C002121
:1010B0000023ECFB0E01FFF723F80121381A03F09F
:1010C000F3FF02F0C1FB0120FFF734FFBFF35B8F9A
:1010D0001D4B0122B24003EB850353E8001F11436F
:1010E00043E800100028F8D1BFF35B8F0C2303FB0B
:1010F000048494E8070005AB83E80700134A1AB19B
:1011000093E8070003F07BFCFFF762FF02F076FD37
:1011100001200F4ABFF35B8F0123B340DB4302EB97
:10112000850555E8002F1A4045E800210029F8D12F
:10113000BFF35B8F08B0BDE8F08100BF4C09002011
:101140003F420F0040420F00EC070020FF49000023
:10115000FC070020F00700200B6801330B60014BF7
:101160001B68184720000020014B1860704700BF23
:101170002000002007B50B460021024601910348DC
:1011800001A9FFF767F903B05DF804FB59110000EE
:1011900008B54FF02002EFF3118382F31288BFF3FA
:1011A0006F8F00F0C5FB034803F0BFFB00F00AF8A7
:1011B000FCE700BFAC550000014910220A607047EF
:1011C00010ED00E072B6404080F31188BFF36F8FDE
:1011D000BFF34F8F30BF62B6BFF36F8F704700BF52
:1011E00072B6494081F3118820BF80F3118862B63E
:1011F000704700BF01B572B60B4A906900281EBF48
:101200000021916103F029FE62B6EFF30580A0F1A1
:1012100010004FEAC0000549014409C99847BDE8DC
:1012200001400349084700004C090020D451000048
:101230002114000030BFFFF7FDBF00BF12498A68CC
:101240004FF030001044EFF3098C80E8F01F2020AD
:1012500080F31288BFF36F8F0C4F4FF00066CA699E
:101260008A603E60506F0023536780F3118804B595
:10127000104600F075FABDE8044002F1300090E835
:10128000F01F8CF3098870474C09002004ED00E042
:101290001EF0040F0CBFEFF30880EFF309808169A3
:1012A00011F8021C0229FFD001B503F05CFB01BD5F
:1012B00043B2002B08DB012200F01F0002FA00F00D
:1012C0005B09024A42F82300704700BF00E100E0DA
:1012D000054B420900F01F0053F82220012303FAB6
:1012E00000F01040704700BF00E100E043B2002B67
:1012F000A8BF03F1604301F10101B8BF064B4FEAFB
:101300004111ACBF03F5614300F00F00C9B2B4BF97
:10131000195483F80013704714ED00E00B4A08B528
:101320000B4B22F07F029A60BFF34F8FBFF36F8F9A
:10133000D3F8882022F47002C3F8882002F098F8CD
:1013400002F0BCFF00F0A0F902F09CF800000000E1
:1013500000ED00E0094A0A4993680968996709495C
:1013600058674B6843F080534B60002383F3118828
:10137000BFF36F8F9368986F704700BF4C090020D0
:10138000C054000000ED00E042F8203C009B42F811
:101390001C3C0A49019B42F8183C029B42F8143C51
:1013A00021F001014FF0807342F8043C42F8081C20
:1013B0000023203A02654367704700BF4F49000091
:1013C0000B4A0346906890B113F1160F406E05D09A
:1013D000A0F120029A4206D8834204D281422CBF57
:1013E0000021012100E00021002908BF00207047F2
:1013F0004C09002008B5094B98600D46144600F0D2
:10140000AFF9204685F30988002163B681F311887E
:10141000BFF36F8F0022002303F099FA4C090020DC
:10142000044B9968D869884203D003494FF0805231
:101430000A6070474C09002004ED00E0EFF30880DB
:10144000EFF3098101B5724600F092F801BD00BFCB
:10145000002080F31488BFF36F8F03F049FE002053
:101460000D490860BFF34F8F0C4880F3088800F0E7
:1014700027F9202080F3118809484FF402614018B1
:1014800080F30988EFF314800221084380F3148865
:10149000BFF36F8FFFF742FF94ED00E08013002051
:1014A0000015002038B5194B14469A6A9A6A9A6A50
:1014B0000546900719D5586B9A6A120615D519B1C9
:1014C0009A6A22F080029A629A6A9A6A9A6AD106A5
:1014D0000ED49B6A9A070BD400200C4A936A43F0FF
:1014E000FF0393620023237038BD6FF01500EBE714
:1014F000064B5B681B05EFD52946FFF761FF002807
:10150000EAD080F309880220E7E700BF00ED00E0A1
:101510000D4B9A6A9A6A9A6A920508D59A6B9A6AEA
:10152000120404D518B19A6A22F400429A62064B5A
:101530009A6A9A6AD20558BF9A6A9A6A002042F457
:101540007F429A620870704700ED00E0074B9A6A8C
:101550009A6A9A6A9A6A9A6A9A6A9A6A6FEA0242D6
:101560006FEA12429A620020704700BF00ED00E06F
:1015700070B53E4B5B688AB00D46C3F30803002686
:1015800086F31188BFF36F8F02F07F41B1F17F4F77
:1015900011D102F00C0108290DD0120701D4054623
:1015A00001260022033B8DF80720032B57D8DFE8E4
:1015B00003F0044E524B3546F3E72C4BDC6A14F033
:1015C00002044CD1DA6A002A18DBDB6A5B0015D50D
:1015D000AB6933F8022C4DF602739A420DD003F139
:1015E000604303F626631B7803B30DF10702012164
:1015F0002846FFF757FF044600E02C689DF80730A7
:1016000093B92022294602A803F0E5F9099B46B3C5
:10161000C3F3080222B96FEA53236FEA4323099305
:1016200002A9204603F09DF90AB070BD104B1B784B
:101630002BB10DF107010120FFF76AFFDBE70D4B2E
:101640001B889BB2002BD9D0FFF780FFD3E70DF1A9
:1016500007020021CCE70DF107010020ECE7002490
:10166000CCE723F4FF7323F00103D8E700ED00E09B
:1016700029ED00E02AED00E0024A536943F010032F
:101680005361704700ED00E0044800232021C21898
:101690000133302B82F80013F9D1704700E100E0EC
:1016A000064A11680023C1F3072118468B4200D176
:1016B0007047936010610133F8E700BF90ED00E0E0
:1016C00008B572B6002383F31388FFF7E9FF144BC4
:1016D0004FF0FF32C3F88020C3F88420C3F888207D
:1016E000C3F88C20C3F89020C3F89420C3F8982046
:1016F000C3F89C20C3F88021C3F88421C3F8882153
:10170000C3F88C21C3F89021C3F89421C3F8982121
:10171000C3F89C2162B6BFF34F8FBFF36F8F08BD34
:1017200000E100E0064B9B68834207D1EFF305839D
:1017300023B1044A536843F08053536002F034BB32
:101740004C09002000ED00E0024B034A0348012150
:1017500000F068B80000042000000020B45300002E
:10176000426E054B203A1A60044A2021C3E9011257
:101770001846012100F060B80008002000000B1599
:10178000F0B51E4F00268E4201DB1046F0BD4468C6
:1017900084B353B104F1FF3C14EA0C0F18D11F2C91
:1017A00016D905681CEA050F12D1202C0568D0F85F
:1017B00008C0D2B20FD9B4F1004F0ED8013CB4FA30
:1017C00084F4C4F11F046400072A4CEA040406D917
:1017D0006FF01502D9E70824F6E73E24F4E725F078
:1017E0001F05154345F0100544F00104BA60FD6083
:1017F00001323C6101360C30C5E700BF90ED00E0DE
:10180000034B05225A60BFF34F8FBFF36F8F7047B2
:1018100090ED00E0BFF35F8F014B00225A607047EC
:1018200090ED00E010B5034C01232278FFF7A8FFEC
:10183000207010BD9C09002008B5084A00231278CA
:10184000FFF79EFF10F1160F03D0054B002207286B
:1018500000DD08BD98601A610130F8E79C0900209E
:1018600090ED00E013490868082810B51ED8FFF76E
:10187000D1FF114C49680022904201F10C0105D1C1
:101880000E4B1870FFF7BCFF002010BDA26051F88E
:101890000C3C23F01F03134343F01003E36051F8A3
:1018A000043C43F0010323610132E5E74FF0FF30D0
:1018B000EBE700BFC053000090ED00E09C09002062
:1018C000014B1860704700BF240000204FF0200338
:1018D000EFF3118183F31288BFF36F8F0F4A012357
:1018E000C2F840354FF08042C2F878350C4A126891
:1018F000082A08D10B4A1268052A04D80A48825CD3
:101900000AB10A4A13604FF080430122C3F88025D0
:1019100081F31188BFF36F8F0020704700E0014012
:101920003001001034010010E4550000380600407A
:101930004FF08043C0B2C3F81C05BFF34F8F054979
:10194000054BCA6802F4E0621343CB60BFF34F8FCC
:1019500000BFFDE700ED00E00400FA0520B1034BF5
:10196000800143F001031847704700BF8053000017
:101970000E4A70B5841AA3100D4C5C430546E4B2C0
:101980000C2000FB04200E464021084403F05EF8C2
:10199000011E05DB074B03EBC40463689847002175
:1019A00028463346BDE87040184700BF1C08002099
:1019B000B76DDBB6F85300002DE9F041104E841BE3
:1019C000A310104C5C43E4B20C256543804605F13E
:1019D00040000F463044402103F051F8011E09DB5E
:1019E000094A7319C3E90E27084B53F83430BDE890
:1019F000F041184740463B46BDE8F041184700BF5C
:101A00001C080020B76DDBB6E14A0000F853000067
:101A1000002270B5012104461046FFF767FC002044
:101A2000FFF746FC0F4800F0EBFE0F4B984215D134
:101A300003F083F926690D49304602F018FF0028AB
:101A40000BDB012535642469084904F11C0002F010
:101A50000EFF002801DBE564002070BD6FF004007C
:101A6000FBE700BFA51A00000000AD0B0854000002
:101A700001460C2309484B4370B5C418D4E90E56EF
:101A800000224033A263184403F017F82DB1324608
:101A90002B460348BDE87040184770BD1C08002065
:101AA0005C51000010B1012804D07047034B1B6C3F
:101AB0005B0701D1FFF7DCBF704700BF1C080020A7
:101AC00008B54FF02003EFF3118183F31288BFF3C1
:101AD0006F8F124A136843F0020013F00103106085
:101AE0000CD04FF08042D2F80C34D2F80C2413F012
:101AF000010303D00A4802F0E0FF012381F31188BB
:101B0000BFF36F8F23B1BDE808400020FFF7B0BFDF
:101B1000BDE80840012000F083BE00BF6C08002033
:101B20005C080020094BBFF35B8F53E8002F22F0C5
:101B3000020143E800100028F7D1BFF35B8FD30701
:101B400002D4012000F09EBE704700BF6C08002048
:101B50001FB500220123CDE90223094ACDF800D0A8
:101B60006B46CDF804D002F0E1FF002805DB4FF40E
:101B700080420023684602F089F905B05DF804FB55
:101B8000FF4A00002DE9F8433A49BFF35B8F064650
:101B9000012251E8003F41E800200028F9D1BFF3BD
:101BA0005B8F33B9344935484B60CB608A6002F0B3
:101BB00071FE731E012B32D8012E07D14FF08043E6
:101BC000D3F81C3403F00303012B28D003F040FAB0
:101BD000044618B92A4B1B78002B44D14FF0200340
:101BE000EFF3118583F31288BFF36F8F0124254F24
:101BF000DFF89480DFF894904FF08042D2F81834E8
:101C0000D2F81824D2030CD503F00303012B01D022
:101C1000012E06D10CB385F31188BFF36F8FBDE899
:101C2000F883ACB12846FFF7DBFA4FF08042D2F8D8
:101C30001835002BE0D139680029DDD03B603B68C6
:101C40000123C2F81835C8F88031C9F80030D3E74D
:101C50000021212002F088F8E7E74FF080430222BC
:101C6000C3F80423DBE74FF080430222C3F80823C4
:101C70000546BCE7700800200C080020380800204A
:101C8000AD0D00200401004000E100E0080000402C
:101C900008B5084B0848186003F0BAF838B107488F
:101CA000FFF70EFE0548FFF75FFA002008BD6FF052
:101CB0001200FBE774080020BC510000C11C0000AA
:101CC0000A2838B5074D044604D1286883680D21D9
:101CD0005B68984728688368E1B25B68984720464C
:101CE00038BD00BF74080020420970B5034602D019
:101CF000012A1DD070BD0F4E326951680029F9D0FC
:101D00000C6803F01F030125002C05FA03F538BF0A
:101D100000248A682A4002D04B6830469847002C3D
:101D2000E8D02368002B38BF002321461C46F0E78B
:101D3000014EE1E7745100008C51000030B540685D
:101D4000047B01F01F05B2F5005F45EA441585B03C
:101D50004FF0000404D1284601F07AF8002032E068
:101D6000B2F5804FCDE902442FD1B3F5003F0CBF4F
:101D7000042305238DF80830836823FA01F1C9078D
:101D80002FD4B2F5A03F2CD16A09012A05F01F0318
:101D90001C4A03F5E07318BF4FF0A04252F82330FD
:101DA000DB071ED40DF107042146284600F0BCFFD6
:101DB000154B984214D1204601F000F8134B98427D
:101DC0000ED06FF00B0005B030BDB3F5C02F05D0BD
:101DD000B3F5003F0CBF02230123CBE70323C9E780
:101DE00003940023194602AA284600F07BFE074B05
:101DF000984204D10121284600F0E6FFAEE76FF0DB
:101E00000400E0E7000300500400AD0B0000AD0B40
:101E100010B500F0C3FF044668B900F097FF084B07
:101E200098420AD10748214600F078FF2246052152
:101E30000620FFF75BFA002010BD6FF00400FBE7FF
:101E40000000AD0BE91C00002DE9F04347683B7B27
:101E500001F01F0585B00E4645EA43151446CAB980
:101E600002A9284600F060FF0446284601F012F857
:101E7000484B984204D06FF0040005B0BDE8F083F1
:101E8000844205D19DF8080000F092FFA042F2D1F3
:101E90000020F2E74FF000090DF103013046CDE9D3
:101EA000029900F041FF4B46804602AA4946284667
:101EB00000F018FE374B984202D06FF01500DCE7B7
:101EC000804503D19DF8030000F072FFA3054ED5B5
:101ED000314B324A234093423AD00CD8062B14D0CF
:101EE00004D893B1022BE8D104230EE0B3F5801F90
:101EF000E3D1012309E02A4A93422BD0B3F5A00F86
:101F00002AD0B3F5800FD8D102238DF8043084F4A1
:101F10008073C3F30023E0068DF8053054BFC4F38B
:101F20004013032321058DF8063017D57B68012166
:101F300001FA06F6C3F80865002201A9284600F058
:101F40007DFE144B984214BF6FF01500002094E7FB
:101F50000723DAE70523D8E70323D6E7620541BF65
:101F60007B68012101FA06F6C3F80C65E4E7E30695
:101F70004FF0000354BFC4F3401403241A4601A9D0
:101F800028468DF8044000F0ADFD024B98423FF426
:101F90007FAF92E70000AD0B0600F00006001000D6
:101FA00002004000F0B54B79012B26D0032B21D144
:101FB00010268B79032B1DD1CC790CB1012C19D1B2
:101FC0000A7912B1022A15D10E220B684568B3F5C1
:101FD000164F2D6865D02DD8B3F5165F64D016D88E
:101FE000B3F5966F62D00AD8B3F5967F61D0B3F59A
:101FF000167F61D06FF0850052E00026D9E7B3F577
:10200000166F5CD0B3F5965FF4D1374B3CE0B3F577
:10201000E14F57D007D8B3F5615F55D0B3F5964F70
:10202000E8D1324B30E047F61227BB42E2D14FF401
:10203000000329E0B3F5613F48D013D8B3F5963FCC
:1020400047D009D84DF6C027BB4244D0B3F5614F05
:10205000D0D14FF46B0317E0B3F5E13FCAD14FF095
:10206000EB7311E0B3F5612F38D008D8204FBB4295
:1020700037D0B3F5E12FBDD14FF0E86304E01D4F39
:10208000BB42B7D14FF08053C5F82435036903C96B
:10209000344322430433C5F86C2583E80300002051
:1020A000F0BD4FF41D03EFE7134BEDE74FF49E2314
:1020B000EAE74FF4A033E7E74FF41C33E4E74FF4CB
:1020C0001D23E1E70D4BDFE70D4BDDE74FF06C73B0
:1020D000DAE70C4BD8E74FF46503D5E74FF07063B0
:1020E000D2E74FF08063CFE700B0130000A04E00AE
:1020F00090D0030040420F000050270000C0750040
:1021000000F03A0000903A0100F01F024009012857
:10211000044B02F5E07218BF4FF0A043890043F86A
:102120002210704700030050F8B5066905460F46B7
:1021300002F08EFF10B92C4B1B7883B94FF02003AF
:10214000EFF3118483F31288BFF36F8F284602F0F8
:10215000A3FD28BB84F31188BFF36F8FEEE76424DF
:10216000284602F099FD70B9012002F0F1FD013C12
:10217000F6D10021212001F0F7FDF0E784F311886A
:10218000BFF36F8FF5E74FF02003EFF3118483F374
:102190001288BFF36F8F284602F07EFD0028EDD035
:1021A00006F8107F69680B680122C3F84465C3F81C
:1021B00048250022C3F82021D3F82001C3F8582174
:1021C000D3F858214A68D20641BF0822C3F8002537
:1021D0004FF48002C3F8042301229A6084F311882B
:1021E000BFF36F8FF8BD00BFAD0D002000F01F02E0
:1021F00040090128044B02F5E07218BF4FF0A043DC
:10220000032143F8221070470003005000F01F0123
:1022100040090128044B4FF0010218BF4FF0A043C2
:102220008A40C3F808257047000300502DE9F041AB
:10223000D0F804800769D8F800400023C4F80035BE
:10224000386045680646E868421C04D0FFF7DEFFA8
:10225000E868FFF7CBFF2869431C06D02B7F002BD3
:1022600014BF03210021FFF74FFF6869421C04D00F
:10227000FFF7CCFF6869FFF7B9FFA869431C06D0D8
:102280006B7F002B14BF03210021FFF73DFFD5E931
:1022900003122B68C3F80C15C3F81425D5E90512F1
:1022A000C3F808153169C3F8102504313046FFF72B
:1022B00079FE0546002846D1D8F80430990719D58B
:1022C00007F1120000F0E2FE224B98423ED1B87CAA
:1022D000C30003F1804303F5F83304F10C0204F565
:1022E0009071C3F81015C3F814251B4A01238340CD
:1022F000C2F804350823C4F8003598F808305BB9F3
:10230000C4F81031D4F8103107F11103C4F8343592
:102310000123C4F838352360D8F804309A075CBF2D
:102320004FF48072C4F80423DB0644BF4FF48003EB
:10233000C4F8043310370023C4F84475C4F8483592
:102340000123A360E3602846BDE8F0816FF0040537
:10235000F9E700BF0000AD0B00F00140194970B56E
:10236000044622F07F460868C1E90023A6F5001361
:10237000101AB3F5400F4FF000050AD2124B19683E
:102380000A060B0A9219114943F10003C1E900231F
:10239000012501F00DFFA30003F1804303F588330D
:1023A000D3F84025B2420BD11DB94FF40002C3F857
:1023B0004025074B4FF4803000FA04F4C3F844433F
:1023C00070BD00BFB801002098080020A0010020C7
:1023D0000010014010B501238340114ABFF35B8F09
:1023E000DC4352E8001F01EA040C42E800CEBEF1D3
:1023F000000FF6D1BFF35B8F4FF4803202FA00F08A
:1024000002F1804202F58052C2F80803BFF35F8FE9
:10241000BFF36F8F0B4214BF0120002010BD00BF1F
:10242000940800200123124ABFF35B8F834052E8D7
:10243000001F194342E8001CBCF1000FF7D1BFF3A5
:102440005B8F0C4A4FF480338340C2F804330A4B4D
:10245000BFF35B8F1B68BFF35B8F23FA00F0C307EA
:1024600042BF064B4FF40032C3F80021704700BF53
:1024700094080020001001409008002000E100E0D6
:102480000D4B1B68190A1806BFF35F8F0B4BD3F86F
:102490000435C01841F10001B3F5801F0AD2084B82
:1024A000D3E90023994208BF904203D210F1807013
:1024B00041F10001704700BF980800200010014062
:1024C000A00100202DE9F04F85B016461F460546B5
:1024D000FFF780FF0190FFF7D3FFB94208BFB0427A
:1024E0007FD2B6EB000867EB010900234FF0807242
:1024F0004B4508BF4245C0F08580444B03EB0513B4
:10250000D3E902239F4208BF964254D04FEA85097F
:102510004FF4803B09F1804905F150080BFA05F2B0
:1025200009F588394FEA88081FFA88F80292384A74
:10253000D9F8400526F07F4308F1804808F588382F
:102540001C469346D2F804A5A0EB0A0020F07F4079
:102550002AF07F410128C9F8401505D103931320C3
:1025600002F0C0FD2A4A039B02990AF1020CA4EB77
:102570000C0020F07F40B0F5000F88BF64460020BB
:10258000C8F80000D8F80000CBF8441324F07F40CE
:10259000C9F84005DBF80405824506D0201A023848
:1025A00020F07F40B0F5000F19D8E41A24F07F44E2
:1025B000321947F10003154C290104EB0510C0E95D
:1025C00002230E9A0F9B625043600024019B13B1BB
:1025D0002846FFF727FF204605B0BDE8F08F2046CC
:1025E000B0E701230B4ABFF35B8FAB4052E8001FFB
:1025F000194342E800100028F8D1BFF35B8F324640
:102600003B46D8E76FF01504E0E700BFA8010020C3
:10261000001001409008002073B5194B194D00249B
:102620004FF0FF304FF0FF31C5F80845C3E9020114
:102630004FF48033C5F80433134B02264FF40032B5
:102640000121C5F804631120C3F880212246FEF75A
:102650004DFE1120FEF72CFE0C4A012313600C4A9C
:102660002B6013600B4B0C4A00930194002320460F
:10267000FFF728FF3046FFF785FA204602B070BD0D
:10268000A80100200010014000E100E00810014016
:10269000940800205D230000FFFF7F002DE9F74331
:1026A000344CD4F804339A0709D5334B1A6832B145
:1026B00000221A60314A1B681368013313604FF01F
:1026C0002003EFF3118283F31288BFF36F8FD4F8E6
:1026D0000433DB0312D5BFF35B8F294B53E8001F94
:1026E00021F0010043E80006002EF7D1BFF35B8F15
:1026F000244B002936D11968002933D1002382F3F5
:102700001188BFF36F8F53B3FFF7BAFE06464FF041
:102710002003EFF3118083F31288BFF36F8F1A4BFE
:10272000D3E90289494508BF46454FF000021ED350
:102730004FF0FF364FF0FF37D3E90015C3E90267CA
:102740001A604FF48033C4F8483380F31188BFF324
:102750006F8F21B1009542464B460020884703B059
:10276000BDE8F083002119601B680123C7E711460B
:10277000EBE700BF00100140041101409808002061
:102780009008002040110140A8010020144B13B50F
:10279000B0F1FF3F08BF1846441E002C1EDD9C42CE
:1027A000A8BF1C46FFF76CFE0E4B0F49D3E9002370
:1027B000801AB0F5000F28BF0024013004440848F7
:1027C0000091844228BF044612194FF00000019086
:1027D00043F10003FFF776FE02B010BD0024E1E7ED
:1027E000FFFF7F00B80100205D23000008B5FFF760
:1027F00047FE024B1B68C01A08BD00BFB80100208D
:10280000044B1A7922B9012218609A800248704755
:10281000024870479C0800200000AD0B0C00AD0B77
:1028200010B1012820D070474FF08043D3F818240E
:10283000D3F8181411F4803F194611D002F00302A6
:10284000012A0DD1C3F818250C4B00221A601B6811
:102850004FF080430222C3F8042301229A6070479C
:102860000023C1F81835EFE7054B00221A601B68FA
:102870004FF08043C3F80403186070470401004020
:102880000001004038B510B1012818D038BD4FF014
:1028900080430222C3F80823184A10601268184ABD
:1028A0000121116042F210751C46D4F81834DB0384
:1028B000ECD5012002F04CFA013DF6D1E6E7114BD0
:1028C0004FF080440022C4F808031A601B680E4BC6
:1028D00042F210751860D4F80C34D4F80C24D203EA
:1028E00003F0010305D523B1012002F031FA013DC7
:1028F000F1D1064B00225A71C8E700BF0401004025
:102900000C00004000010040040000409C08002032
:10291000164B1A6810B56AB100221A601B684FF096
:1029200080430122C3F80823114B587910B95A711A
:102930001B6898470F4B1A6872B100221A601B6817
:102940004FF08043D3F81824D3F81814920704D119
:102950000122C3F818259A6010BD0222C3F808238B
:10296000034BBDE810401B680120184700010040E0
:102970009C0800200401004070B501250368B3FAEB
:1029800083F2202AC2F11F0414D0BFF35B8F05FA33
:1029900004F223EA020250E8006F9E4204D140E8AC
:1029A000002CBCF1000FF6D1BFF35B8FE6D10248DB
:1029B0000C7070BD0148FCE70000AD0B0200AD0BD0
:1029C0000368CB40DB0710B515D4012303FA01F1EE
:1029D0000368BFF35B8F41EA030250E8004F9C425B
:1029E00004D140E8002CBCF1000FF6D1BFF35B8F9F
:1029F000EED1024810BD0248FCE700BF0000AD0B5D
:102A00000400AD0B036803F01F025B09012B026099
:102A1000024818BF4FF0A040704700BF00030050AD
:102A200070B500F108030C4C34F81330DA05054694
:102A30000E4607D5C3F3432304EBC30254F83330E7
:102A400052689847A3682BB1E26831462846BDE832
:102A50007040184770BD00BF50000020124B083076
:102A600010B433F81020D1051BD5C2F3432122F452
:102A7000F85223F8102003F11004002034F8022B40
:102A800012F4807F03D0C2F34322914209D0013077
:102A90003028F3D1002243F83120044810BCFFF75E
:102AA0008FBF10BC704700BF50000020C400002042
:102AB00038B50A4C00F1080534F815309A0606D5E9
:102AC0005B0B074A03F5A273002142F82310FFF7BE
:102AD000C5FF002324F8153038BD00BF500000208A
:102AE000006000402DE9FF411D46044617460B4695
:102AF00009B34D4E00F1080836F8182002F0220202
:102B0000222A03D1494804B0BDE8F0810022CDE972
:102B100000228DF80E208DF80F200DF10E010DF121
:102B20000F0202F017F936F8183023F0020343F0D1
:102B3000010326F8183097B13B483E787A6804F1D3
:102B4000080330F813108F070CD5002ADAD130F8BB
:102B5000132022F01C0242EA860220F81320CDBB8B
:102B60003348D0E721F02001C904C90C20F8131024
:102B7000002AECD0032EC5D817782EB92D4A07F5B8
:102B8000A27142F82160E2E7BA0002F1804202F548
:102B9000C0424FEA042ED2F810C52CF0030CC2F844
:102BA00010C5D2F810C52CF44F3C2CF4407CC2F870
:102BB00010C5D2F810C50EF47C5E4CEA064C41EA12
:102BC00047314CEA0E0C41F0200120F81310C2F8F6
:102BD00010C5BCE7D5E900672046FFF73FFF002E90
:102BE000BED0114D2B689E4204D16B689F4201D12B
:102BF000002209E010480DF10F01FFF7BDFE0C4B5C
:102C0000984280D19DF80F2045F8326005EBC20351
:102C100008345F6035F8143043EA422343F480738C
:102C200025F814309CE700BF500000200400AD0BD5
:102C30000000AD0B00600040C4000020F0B5044669
:102C400085B0154609B300F10807314E36F8173044
:102C5000980701D49A0658D413F01C0F02D04B7871
:102C6000012B52D001238DF80F300023CDE9001342
:102C70004A1C8B1C20460DF10F0102F06BF836F850
:102C8000173043F0030326F8173015B9214805B073
:102C9000F0BD1F4E04F1080736F81700830734D53E
:102CA00095F800C06146890020F0200001F18041C4
:102CB000C00401F5C041C00C26F817000023C1F87C
:102CC00010356A78002AE1D0D1F81035AD7823F4B8
:102CD000991323F4F853C1F81035D1F810E5230205
:102CE00003F47C53120443EA0E0302F440322D0530
:102CF000134305F4801540EA4C302B4340F020008C
:102D000026F81700C1F81035C0E70348BFE700BF39
:102D1000500000200000AD0B0400AD0B014BC3E9D7
:102D200002017047500000200830054B33F8103086
:102D30009A0643BF5B0B03480B700348704700BF04
:102D4000500000200000AD0B0400AD0B38B50E4C58
:102D500094F87850B5B96022294604F1100001F0CA
:102D600045FE0620FEF7A4FA084B09481D601B68C3
:102D7000084B4FF00042C3F80423012384F8783055
:102D8000636738BD0448FCE7500000207C610040C8
:102D90000000AD0B006000400500AD0B034B93F845
:102DA0007800003818BF0120704700BF5000002095
:102DB00001460148FFF704BEC0000020014601485B
:102DC000FFF7DABDC000002037B51F4B00F1080245
:102DD000044633F812309A061DD513F002051AD1B5
:102DE0005B0B9A0002F1804000F5C24002F1804284
:102DF00002F5C04205600068D2F8100540F00100FD
:102E0000C2F8100529B1012202FA03F30F4AC2F8F1
:102E1000043303B030BDC3F38203042B10D0052B61
:102E200010D001A80194FFF7EDFD019BD0F810151B
:102E3000D94001F001010231204601F0D2FFE8E75C
:102E40000321F9E70221F7E750000020006000406D
:102E50000E4B00F1080233F81230990613D59A0789
:102E600011D45B0B01229A409B00094903F1804376
:102E700003F5C043C1F80823D3F8102522F003025C
:102E8000C3F810257047002101F0ABBF50000020AF
:102E9000006000400E4B00F1080213B513F8123029
:102EA000DB07044611D5FFF7D3FF2046FFF700FEEE
:102EB00001A80194FFF7A6FD019B03F5E073022230
:102EC00040F82320034802B010BD0348FBE700BFD1
:102ED000500000200000AD0B0400AD0B2DE9F04FB9
:102EE000644B65486549002587B001222C461E6861
:102EF00036B1D0F8046316421EBF1C601E6815432D
:102F000004338B424FEA4202F1D15D4F3B687BB301
:102F10004FF0A0435B4ED3F820250492C3F8202540
:102F2000D6F820350593C6F8203500960DF1100926
:102F30004FF000084FF0010BD9F80030F3B908F159
:102F40002008B8F1400F09F10409F5D13B603B6856
:102F500000994FF0A043D3F820250492C3F8202510
:102F6000009BD3F820350593C1F820351343DDD1FC
:102F70000124002D66D107B0BDE8F08F93FAA3F3CA
:102F8000B3FA83F308EB030606F108023E4B0396FF
:102F900033F81220C2F38203F40801939A4604AB7B
:102FA00006F007000BFA00FC185D20EA0C0018552B
:102FB00003A89108FFF726FD039C04F5E0744B0776
:102FC00050F82440C4F3014423D551463046FFF75E
:102FD00027FD03A80396FFF715FD039A02F5E0729B
:102FE000E4B250F82220C2F30142944207D10021FA
:102FF000304601F0F6FE2146304601F0F2FE03A80D
:103000000396FFF7FFFC039B0BFA03F3C0F8203590
:1030100092E7022C0CBF03210221304601F0E1FEB1
:10302000019B032B04D0022C07D1BAF1010FE6D18A
:1030300051463046FFF7F4FCE1E7032CDFD1BAF14B
:10304000020FF4E795FAA5F3B3FA83F304FA03F257
:103050009B0003F1804303F5C04325EA0205D3F842
:103060001005D3F81015C0F30520C1F30141FFF797
:10307000D7FC7EE700610040006000402061004016
:103080007C610040000300505000002001460148D0
:10309000FFF772BCCC000020034B1868A0F10803B6
:1030A00058425841704700BF30010010064B1B6862
:1030B000082B06D1054B1B68052B02D8044AD05CAF
:1030C00070470020704700BF30010010340100102D
:1030D0000B560000024AD2F80034002BFBD0704798
:1030E00000E0014010B5FFF7D7FF40B14FF080433B
:1030F0000022C3F80C21C3F81021C3F83825FFF7CC
:10310000CBFF002846D04FF080525B4BD2F804141E
:10311000C3F82015D2F80814C3F82415D2F80C14FB
:10312000C3F82815D2F81014C3F82C15D2F81414CB
:10313000C3F83015D2F81814C3F83415D2F81C149B
:10314000C3F84015D2F82014C3F84415D2F824145B
:10315000C3F84815D2F82814C3F84C15D2F82C142B
:10316000C3F85015D2F83014C3F85415D2F83414FB
:10317000C3F86015D2F83814C3F86415D2F83C14BB
:10318000C3F86815D2F84014C3F86C15D2F844247B
:10319000C3F87025FFF78AFF10B1384B384A1A6020
:1031A000FFF784FF18B1374BFB22C3F81825FFF750
:1031B0007DFF48B13449354B0A681B6822F00F0285
:1031C00003F00F0313430B60FFF770FF18B1304B90
:1031D0004FF400721A60FFF75FFF48B14FF0804371
:1031E000D3F80024D20744BF6FF00102C3F80024D3
:1031F000284B1B68082B0ED1274B1B68052B02D8C8
:10320000264AD35C3BB14FF01023D3F808224FF08D
:103210008043C3F858254FF01023D3F80022002A2A
:1032200003DBD3F80432002B22DA1D490123C1F855
:103230000435FFF74FFF4FF010201224C0F8004272
:10324000FFF748FFC0F80442FFF744FF0023C1F82E
:103250000435FFF73FFFBFF34F8F1249124BCA6887
:1032600002F4E0621343CB60BFF34F8F00BFFDE772
:103270000E4B0F4A1A6010BD00C000408C56004033
:103280004881030000F00040E40E004058020010A6
:103290004096024030010010340100100556000035
:1032A00000E0014000ED00E00400FA05D00000203D
:1032B0000090D00310B5144C144A15490323236120
:1032C0006361144BA261E3614FF4806323620023C6
:1032D000A3626362E36222660F4A6266E01D102207
:1032E000A2662367E366636701F04FFBBFF35F8F5E
:1032F0000A49204601F049FBBFF35F8F2023A371E9
:10330000BFF35F8F10BD00BFA4080020115600005E
:103310001A560000AD0900209D0900201E5600002D
:103320000E4B70B553F82040013053F82060A64290
:1033300000D870BDD4E900352846984765B1EB68E0
:1033400030B10028B8BF4042FF28A8BFFF20187046
:103350005A7842F001025A700834E8E7AC54000091
:1033600070B5054610B90024204670BD0378002BC7
:10337000F9D00F4A0F4C1646944208D10D4CB44276
:10338000F1D0204601F044FD50B91834F7E720464B
:1033900001F03EFD10B12368AB42E5D01834EBE7F5
:1033A0002168284601F00BFB0028EED1DCE700BFC6
:1033B000D45100005C51000008B5094C4FF02002C8
:1033C000EFF3118382F31288BFF36F8F01F05CFE7D
:1033D000A061FDF741FE0028F0D1FDF7F3FEEDE717
:1033E0004C09002030B5002387B00122CDE9042329
:1033F0000F22CDE902320D4C0D4A01930D491823DD
:1034000004EBC01403FB00234FF4B075009305FBDD
:103410000011094B4FF4A072204600F061FD637B60
:1034200023F00403637307B030BD00BFC001002068
:103430004C090020A0130020B933000008B50A4B46
:10344000012202201A70FFF76BFF00F051FF0320EA
:10345000FFF766FF00F076FDFCF7CCFF034A137B15
:1034600023F00103137308BDAD0D002040020020BE
:103470000248034A0021121A01F0B8BAA001002044
:103480006C0F002080B5DFF8D880A6B088F30888DC
:103490002D4D2E4E6B69DFF8CC9043F40073002461
:1034A0006B61E02385F82230EC772C766C76AC7675
:1034B00085F820406B6A43F4E0236B6285F8234073
:1034C000FEF7DAF8FDF778FE4FF0FF33AB62EB6200
:1034D000FEF7C8F9FEF738F940F20113ADF82430D1
:1034E00006ABB360CDE91F4401F091FC2046FFF725
:1034F00017FF0120164DFFF713FF00F09BFB154B44
:103500000593012314490094CDE903434FF48062ED
:103510004B46CDE901442846F56100F0E1FC6A7BA9
:1035200022F004026A730746284601F01AFD20467D
:10353000FFF758FF094BF3604A4639462846347571
:10354000C6F80480FDF756FF00ED00E04C090020AE
:103550004002002025560000800F0020C0010020FE
:10356000201D00203D34000070B50E4B0E4CA342D0
:1035700001D3002070BDD3E9030141EA000212F03B
:1035800003020BD19D685A61AA4201D11C33EEE7B8
:103590005E690E60013259610144F5E76FF0150074
:1035A000E8E700BF5001002050010020D3B50C46D1
:1035B00016461F464FF02003EFF3118183F3128864
:1035C000BFF36F8F43695BB123601B6843618369FD
:1035D00001338361002081F31188BFF36F8F11E005
:1035E00056EA070203D123606FF00B00F3E70246AF
:1035F000CDE90067083000F06FFA18B9024B9B68FC
:103600005B69236002B0D0BD4C0900202DE9F34175
:10361000044616461F464FF02003EFF3118883F34C
:103620001288BFF36F8FC368354A6BB180689168A9
:10363000884219D056EA070318D188F31188BFF3DE
:103640006F8F6FF00F000CE0916891F90E102161FF
:103650000133E3609368A36088F31188BFF36F8F31
:10366000002002B0BDE8F0812169F0E791F90E1069
:1036700090F90E309942A8BF19466FF07E02914230
:10368000B8BF11468B422FDD00F03AFA0546CDE96E
:1036900000671C482246414600F01EFA0028E0D090
:1036A0004FF02003EFF3118683F31288BFF36F8F7F
:1036B000236821699C420AD04BB193F90E3099429C
:1036C000A8BF19466FF07E039942B8BF1946A0689B
:1036D00090F90E30994209D16DB10A48314600F097
:1036E000A1F86FF00A00BCE70025D0E700F008FA67
:1036F0000028F2D1F0E786F31188BFF36F8FF0E76F
:103700004C090020AE0D002038B583680446002B1C
:1037100036D01E4A9268934235D1DA7B013ADA7389
:10372000C368012B05D9013BC36000F067FA002094
:1037300038BD4FF02003EFF3118583F31288BFF3F8
:103740006F8F0169806890F90E30994201D000F0C6
:10375000D7F9204601F064FCA06058B190F90E2022
:1037600022610022826701F0FCFB0948294600F033
:1037700059F8DAE7E06085F31188BFF36F8FD4E77B
:103780006FF01500D4E74FF0FF30D1E74C0900206F
:10379000AE0D002010B5084C23685BB1FFF726F88A
:1037A00003462068054A0344BDE810401361002128
:1037B00001F07ABC10BD00BF7C0900204C0900203C
:1037C000F8B504460D464FF02003EFF3118683F35E
:1037D0001288BFF36F8F104B00224FF4004740F266
:1037E000E73000211A61E7FB040100234FF47A72ED
:1037F000FCF786FC002C094B09DC1860084B1D60A7
:10380000FFF7C8FF86F31188BFF36F8FF8BD02285A
:10381000B8BF0220F1E700BF4C0900207C0900205E
:103820007809002049B9EFF3058030B9054BDA6912
:103830009B689A4201D0FDF78DBD81F31188BFF3DB
:103840006F8F70474C0900204FF02003EFF3118178
:1038500083F31288BFF36F8F044B9A68D37B013BCD
:10386000D37381F31188BFF36F8F70474C09002029
:1038700038B502460C480D4D01F069FB044600B90D
:10388000EC68AB684AB95A7BD20606D1A26922B964
:10389000DA897F2A01D9EB6138BD9C4201D0FFF75C
:1038A00079FFEC61F8E700BF6C0900204C090020AB
:1038B00070B590F90D20437B002A014604DA03F02D
:1038C0007F03437301F01BFB4B7B174A63F07F03BD
:1038D00010464B7350F8203F556A834208BF0023BF
:1038E000002B38BF0023CBB191F90E6093F90E4045
:1038F000A6420FD0A41B002C0CDD5868C1E9003093
:10390000016059609068431A5842BDE870405841C0
:10391000FFF7AEBFAB4201D01B68E4E7C1E9000589
:1039200029605162EEE700BF4C09002070B50146E6
:103930004FF02003EFF3118483F31288BFF36F8FEE
:10394000164B174A98681568A8421D4606D1FFF71E
:1039500021FF84F31188BFF36F8F70BD00261660BE
:10396000104A1268BAB1C2897F2A14D8427BD206A3
:1039700011D10D4A90F90E60126896420BDB0B4A8A
:10398000904208D01A698A4202DCFFF791FFDEE715
:10399000521A1A61DDE700232B61DAE74C09002097
:1039A000740900207C09002078090020C001002053
:1039B00070B490F90D30427B002B2DDBD3062BD158
:1039C00083694BBB154962F07F0242730A464D6A18
:1039D00052F8204F944218BF2346002B38BF0023D3
:1039E000ABB190F90E6093F90E40A6420BD0A41B28
:1039F000002C08DD5A68C0E900321060586070BCC5
:103A00000020FFF735BFAB4201D01B68E8E7C0E9F3
:103A1000002528604862F2E770BC70474C0900201E
:103A200010B54FF02002EFF3118482F31288BFF338
:103A30006F8F427B510704D484F31188BFF36F8FDB
:103A400010BD22F004024273FFF7B2FF2146024884
:103A5000BDE81040FFF7E6BEAE0D002008B590F9B6
:103A60000D20437B002A014604DA03F07F034373F1
:103A700001F045FA044B9868431A58425841BDE892
:103A80000840FFF7F5BE00BF4C0900202DE9F041CA
:103A9000064614461D464FF02003EFF3118783F3CB
:103AA0001288BFF36F8F01F08EFA87F31188BFF38E
:103AB0006F8F6B1C08BFB4F1FF3F08D022462B4626
:103AC00006F118000349BDE8F04100F0E9BABDE88D
:103AD000F08100BF834F000010B5074B9868074B7B
:103AE0000C4618601146DDE90223FFF7CFFF2046A0
:103AF000BDE81040FDF72EBC4C09002074090020E1
:103B0000F8B504464FF02003EFF3118683F31288D3
:103B1000BFF36F8F437BDA0649B238D18569002D38
:103B200035D103F07F03437301F0E9F9437B8173DF
:103B300063F07F0343731748034653F8207F9F4287
:103B400018BF3D46002D476A1A462B4638BF002352
:103B5000C3B193F90E50A94210D06D1A002D0DDD9E
:103B60005A68C4E9003214605C600120FFF780FEEF
:103B7000012086F31188BFF36F8FF8BDBB4201D0DF
:103B80001B68E5E7C4E900273C604462EDE7A173E8
:103B90000020EEE74C09002070B50446183001F013
:103BA0005DFA4FF02003EFF3118683F31288BFF321
:103BB0006F8F94F90D20637B002A05DA03F07F03F1
:103BC0006373204601F09BF90B4D637BA86843F0BB
:103BD00010036373031B58425841FFF749FE86F3F5
:103BE0001188BFF36F8FAB68A34203D1BDE870406B
:103BF00001F0A3B970BD00BF4C09002010B54FF013
:103C00002003EFF3118483F31288BFF36F8F084B07
:103C10009A68D37B0133D3730020FFF729FE84F326
:103C20001188BFF36F8FBDE8104001F086B900BF67
:103C30004C090020044B002103F12002C3E90822B3
:103C40000846FFF7BDBD00BF4C090020F8B54FF096
:103C50002003EFF3118483F31288BFF36F8F1B49A6
:103C60008868437B03F07F03437301F048F98A6857
:103C7000537B084663F07F03537350F8203F4E6A2E
:103C8000834208BF0023002B38BF0023CBB192F939
:103C90000E7093F90E50AF420FD0ED1B002D0CDDCE
:103CA0005968C2E900310A605A600120FFF7E0FD5F
:103CB0002046BDE8F840FDF74DBBB34201D01B687C
:103CC000E4E7C2E9000632604A62EEE74C090020F0
:103CD0002DE9F04104460D4654EA050104D1FFF7F1
:103CE000B5FF0020BDE8F0816FF001010A1A4FF026
:103CF000FF3161EB0503012A73F100032ADA01F0B9
:103D0000EDF906194FF02003EFF3118883F31288C1
:103D1000BFF36F8F114F124BB8681860FFF79EFE0C
:103D2000B868104922462B46183000F0B9F9BA6835
:103D3000537B43F0100353734046FDF70BFB01F038
:103D4000CDF9301A66EB0601012871F10003B8BF06
:103D50000020C7E76FF00106361AD3E74C090020B0
:103D600074090020834F000008B50B46013308BFDB
:103D7000B0F1FF3F06D1084B9868FFF70DFF4FF0F9
:103D8000FF3008BDFFF7A4FF4FF47A7380FB0323D5
:103D9000D00B40EA4340F4E74C090020014B9868FF
:103DA000704700BF4C0900202DE9F04104464FF058
:103DB0002003EFF3118683F31288BFF36F8F437BE9
:103DC0001A0705D586F31188BFF36F8FBDE8F08120
:103DD00023F0200242F00801D20920D14173A368E8
:103DE00013B1204601F093F804F1180001F036F900
:103DF00004F158074FF00008A56DBD4200D0B5B9D9
:103E00000120FFF735FD104B9B68A342DAD1EFF399
:103E10000583002BD6D13046FDF79CFAD2E703F09C
:103E20005F0343F00803437301F069F8D7E72846BE
:103E300001F06DF805F1180001F010F9C5F878806F
:103E40002846FFF7B5FDD7E74C09002038B50446F2
:103E50004FF02003EFF3118583F31288BFF36F8FC8
:103E600001F0DEF848B10022826701F07AF82946B5
:103E70000548BDE83840FFF7D5BCD4E902329A4284
:103E800018BF0133A360F2E7AE0D002037B514462A
:103E90001D464FF02003EFF3118183F31288BFF327
:103EA0006F8F836843B1013B836081F31188BFF357
:103EB0006F8F002003B030BD54EA050306D181F3B3
:103EC0001188BFF36F8F6FF00F00F3E70246CDE963
:103ED00000450248FFF700FEECE700BFAE0D0020F2
:103EE0002DE9FF410E9E0673042646730D9E8673D0
:103EF00000F158050F46D61DC0E916550C9A00254D
:103F000026F007062037C0E90655C0E91976856016
:103F1000C573C56606F1200802920B9A0192884487
:103F20000A9A009242460446FDF72EFA044B656554
:103F30009B6803B11B6F2367404604B0BDE8F08166
:103F40004C0900202DE9F0472A4E2B4D86B0B04693
:103F5000B54205F1300410D3FFF776FC264CDFF8AC
:103F60009CA04FF4004940F2E7360027444521D396
:103F700006B0BDE8F047FFF741BE54F8043C059396
:103F800054F8103C049354F8143C039354F8183C30
:103F9000029354F81C3C019354F8203C009354E9DC
:103FA0000A2354E90C01FFF79BFF54F8303C5D6590
:103FB0002546CDE7636A5A1C0DD023EAE3733046E9
:103FC0003946C9FB0301B94208BFB042256804D194
:103FD0002846FFF725FD3034C8E74FF47A720023F6
:103FE000FCF78EF802460B4605F11800514600F02A
:103FF00057F8F0E75001002050010020834F0000E7
:10400000034B1B680BB9FEF7F1BB0020704700BFE4
:104010008009002030B5036868B10A4A52689042AE
:1040200009D043B1D3E90421D0E90445121945EB85
:104030000101C3E90421426813605A600023C0E90A
:10404000003330BDD400002038B5134B1C689C42AF
:1040500008BF0024FFF7D4FF0546BCB1D4E9040132
:10406000401B61EBE571012871F1000311DB6FF07A
:1040700000420023824273EB010400DA1046074B32
:104080001B6913B19842A8BF184638BD6FF00040B5
:10409000F5E70020F3E700BFD40000204C09002022
:1040A000B3F1FF3F08BFB2F1FF3F2DE9F74F0446E0
:1040B00092469B4673D081604FF02003EFF3118549
:1040C00083F31288BFF36F8F6FF00103B3EB0A081D
:1040D0004FF0FF3262EB0B09B8F1000F79F10001EC
:1040E0001CDB3048D0E900105B1A62EB0002B3EB36
:1040F0000A0662EB0B07012E77F10003BCBF012615
:104100000027C4E90467284AD2E9003C93421ED143
:10411000C4E9002CCCF8004054602DE0FFF770FF9C
:104120001AF1010300934BF100030193DDE9002331
:10413000121843EBE073C4E90423E4E7B6EB08008C
:1041400067EB09016345C4E90401E1D01B68002B5A
:10415000DED0D3E90489D4E90467464577EB090149
:10416000ECDAB8EB060069EB0701C3E90401596812
:10417000C4E900310C605C60136893420BD09C4230
:1041800009D1FFF761FF18B1084B1B69834202D0C8
:104190000021FEF7FBFA85F31188BFF36F8F03B0A0
:1041A000BDE8F08FC0020020D40000204C090020A0
:1041B0002DE9F74F0646FFF7B9FB4FF02003EFF369
:1041C000118483F31288BFF36F8F2C4DDFF8B0A0FA
:1041D000DFF8B0B02E605146D5F800C0DBF8000023
:1041E0006246D3175845DAE90089CDE900230DD09E
:1041F00060B1D0E90467B445BB411EDA009BB6EB61
:10420000030C019B67EB0306C0E904C6009B13EB9C
:104210000802019B4FF0000643EB0903C1E90023AC
:104220002E60FFF711FF3146FEF7B0FA84F31188D4
:10423000BFF36F8F03B0BDE8F08F18EB06084FF0A7
:1042400000024FF0000349EBE679C0E90423ACEB30
:104250000606CAE900892E60FFF7DCFE84F31188A8
:10426000BFF36F8F836898474FF02003EFF31184FB
:1042700083F31288BFF36F8F0149ADE780090020F7
:10428000C0020020D400002010B54FF02003EFF34F
:10429000118483F31288BFF36F8FFEF7A7FA064BE2
:1042A000D3E90023121843F1000384F31188BFF30C
:1042B0006F8F1046194610BDC002002008B5064891
:1042C000064A0749121A00F086FBBDE80840054A75
:1042D0000549064800F07FBB00000020A001002037
:1042E0006056000000000000605600000000002042
:1042F000024A0349034800F018BB00BF5F560000A4
:104300002A5600003956000010B50A4C23681BB12C
:1043100001232360002010BD00F0D6F80028F7D05C
:104320000138062803D8044B53F8200010BD034879
:1043300010BD00BF84090020C4540000FE8FFFFFA1
:10434000BFF34F8F0549064BCA6802F4E06213437E
:10435000CB60BFF34F8F00BFFDE700BF00ED00E073
:104360000400FA05F0B4094F094E0A4C0A4A0B4DF5
:104370000B494FF0FE333B605268336023600024EA
:104380002B60C1F80045F0BC104700BF00B40250DC
:1043900004B4025008B40250DC0000200CB40250F7
:1043A00000A00250D0E90012014BC3E9001270478F
:1043B000DC00002010B5044630B16368DB0602D58E
:1043C00000232360636010BD024B03485B6898477D
:1043D000F3E700BFDC000020E054000068B1436850
:1043E0003BB1DB0607D5BFF35F8F002303601846A0
:1043F000704703487047034870476FF4E0407047C8
:10440000EA8FFFFFE98FFFFF10B5044620B10022BD
:1044100011232260636010BD0148FFF7A3FFF6E798
:1044200008550000C0B14368A3B1DB0610D50122D6
:10443000BFF35B8F50E8003F40E800210029F9D12D
:10444000BFF35B8F012BF3D0BFF35F8F002070476A
:1044500003487047034870476FF4E040704700BF5F
:10446000E98FFFFFEA8FFFFF70B5D0E90023134CFF
:10447000134DC4E90023D0E90263C4E90263114B80
:10448000086818604868586088689860D1E90360D7
:10449000D5F81411DE601861CB060DD50023C5E9EF
:1044A0004433C5E96D3305F588709047236805F5F9
:1044B000DA70BDE87040184770BD00BFEC00002006
:1044C000B00D0020FC00002010B500F033F820B142
:1044D000032400F067F8204610BD00F035F890B9CD
:1044E00000F0B0F890B90F4B1B681B0EF02B08D1F1
:1044F0000D4A0E4B12689A420AD0072400F01CF8AD
:10450000E7E70624FAE70424204610BD0024F5E777
:10451000012000F097F804460028F7D1044B1860FA
:10452000D9E700BF28B9025024BA02500000E020A9
:104530000CBA02500020704700207047014B1860F1
:10454000704700BF04BA025010B5114800F048F897
:1045500000B110BD0F4800F043F80028F9D10E4C0F
:10456000204600F03DF80028F3D10C4B0C481C60AD
:1045700000F036F801460028EBD100F02DF8044693
:1045800008B1204610BD00F03FF82046FAE700BF12
:1045900034010020280100203001002038010020D3
:1045A0002C01002008B5084800F024F8074800F066
:1045B00021F8074800F01EF8064800F01BF8BDE897
:1045C000084000F00BB800BF340100202801002093
:1045D000300100202C01002000207047704700BFF0
:1045E00008B5034B02681B6810689847002008BD97
:1045F000EC00002008B5034B02685B681068984720
:10460000002008BDEC00002070B5094C094D206960
:10461000AB68984718B1084B08485B689847084A48
:10462000EB68206900211160BDE87040184700BFA9
:10463000FC000020EC000020DC0000202C550000D5
:104640009809002070B51A4D1A4E0446B2682869C0
:104650009047F0B95CB1184C2368ABB1012B1AD06C
:10466000013B23602869F3689847002070BD124C15
:10467000216839B9114B124A0120C3F800051368AB
:10468000002BFCD101312160F36828699847002094
:1046900070BD0C4870BD0A4A1368002BFCD1074A54
:1046A0006FF07E40C2F80035FFF748FF2368D7E778
:1046B000FC000020EC0000209809002000A002501F
:1046C00010B90250E98FFFFF2DE9F74F9946D378D3
:1046D00014466F2BA3F1410206460F4601922DD0DE
:1046E00028D8582B14BF0A251025DDF83080AA469B
:1046F0004FF0000B52465B4630463946FBF700FD53
:10470000092AD3B21FD830335F45DBB208BF564504
:1047100008F8013D01D3C84512D823789B0605D57A
:10472000082D16D1A37843F00803A370404603B0C8
:10473000BDE8F08F03F0F703702BD3E70825D4E72B
:1047400006460F46D6E7019A192A94BF37335733E6
:10475000DAE7102DEAD1A37843F01003E5E72DE95D
:10476000F0410746884615461E461446B442A4EB5F
:10477000050002D33EB923782BB114F8010B414652
:10478000B8470028F2DABDE8F0817047034658B117
:10479000426802F00302012A03D0032A04D102680E
:1047A00012B10020986070476FF0150070474268A2
:1047B000816002F00302032A4FF0000203460CBF9F
:1047C000006810465A60704708B50020FCF7E0FC0E
:1047D000038B13F0070305D10368002B0CBF0020E7
:1047E00003207047022B05D1438B002B14BF002000
:1047F00004207047012B05D10368002B0CBF00205B
:1048000005207047002070472DE9F0410D4607460E
:104810001946281D90461E46FFF7C9FF044638B1C9
:104820003346424629463846A446BDE8F041604733
:10483000BDE8F08110B44FF02004EFF3118284F34F
:104840001288BFF36F8F416110BC0121FCF78CBA55
:1048500010B50C4640B139B1081DFFF797FF28B9D4
:10486000A36833F0030301D06FF0150010BD38B515
:104870000C46054658B151B10B6843B14B6833B192
:104880001C22002100F0B2F82C61002038BD6FF02E
:104890001500FBE770B504460E46FFF7D9FF051E6D
:1048A00031DB4FF02003EFF3118183F31288BFF364
:1048B0006F8F638B208B4FF6FF75AB4200F00702C2
:1048C0002ED0022A0ED1013363831546012381F3D2
:1048D0001188BFF36F8FB3B1002331462046FFF735
:1048E00093FF10E0830701D0062A0ED10023336026
:1048F000636893B9C4E90066154662B90A46204662
:104900000221FCF731FA284670BD052A0CBF6FF072
:1049100085056FF004050023D9E71E606660EBE7AC
:104920006FF00A05F7E7002070470FB407B504A938
:1049300051F8040B0191FCF71DFC03B05DF804EB8A
:1049400004B070470022C0E900228260704704462C
:1049500008B5084611461A46A047FFF71FFAFCF7AC
:10496000E1FE00F05FBA0146006800F05BBA00218A
:104970000120FFF7F6BF08B5FCF75CFCBDE8084076
:10498000FCF74EBD4FF0FF3070470139034611F878
:10499000012F0AB91A70704703F8012BF7E7034695
:1049A00000201A5C02B970470130FAE70346002084
:1049B0001A5C0AB1884200D170470130F8E7431E03
:1049C000013913F8012F11F8010F824201D1002A99
:1049D000F7D1101A704710B5431E0A44914200D116
:1049E00010BD11F8014B03F8014FF7E7C9B20244BB
:1049F0000346934200D1704703F8011BF9E784B0E6
:104A000004AB03E907009DF80430062B08D14FF0F2
:104A100080430122C3F80025BFF34F8F20BFFDE77D
:104A200004B0704784B004AB03E90700002383F3AC
:104A30001188BFF36F8F04B070470269CBB20C21AD
:104A400003FB0121086C00F0070070474FF02003C2
:104A5000EFF3118283F31288BFF36F8F036813F0B3
:104A6000C00301D08B4207D101230360002082F3F1
:104A70001188BFF36F8F70474FF0FF30F7E710B525
:104A80004FF02003EFF3118283F31288BFF36F8F8F
:104A9000036803F00704012C06D10160002082F3B3
:104AA0001188BFF36F8F10BD03F0C0038B4214BF9A
:104AB0004FF0FF306FF07700F1E74FF02003EFF396
:104AC000118283F31288BFF36F8F036803F0C00372
:104AD00043F00203036082F31188BFF36F8F7047C6
:104AE000006910B4CBB21C2403FB0400002110BCED
:104AF00010470020FDF794BE0020FDF7C3BE10460E
:104B0000FFF7A4B938B5CCB20C230546634300695E
:104B1000403380211844FFF799FF002805DB6968BE
:104B200001EBC40463689847002038BD2DE9F843C1
:104B3000CDB20C2704696F43064607F1400080217F
:104B4000204490469946FFF79AFF002807DB3C4433
:104B5000C4E90E89736853F8353098470020BDE8E2
:104B6000F88343685B68D3F810350B60002070470A
:104B700043685B68D3F8040542400A404240C3F8EA
:104B800004250020704743685B680020C3F80815BF
:104B9000704743685B680020C3F80C157047436892
:104BA0005A68D2F804354B40C2F8043500207047EB
:104BB0000369586830B558B10024814213D10868A0
:104BC0005CB99C685860A14200D1986000200860E0
:104BD00072B9002030BD2846EFE720609868814216
:104BE00008BF9C60F2E705680446002DF3D13AB196
:104BF0005A680A60986859600028EAD19960E9E724
:104C00006FF01500E6E743681B68D3F80423D1056D
:104C100018D5D3F82021AAB14FF02001EFF311826B
:104C200081F31288BFF36F8FD3F8201131B10021C7
:104C3000C3F82011D3F820110121D96082F3118823
:104C4000BFF36F8F42685268D20615D54FF020012E
:104C5000EFF3118281F31288BFF36F8FD3F85811ED
:104C600011B10021C3F800154FF48001C3F80813F7
:104C700082F31188BFF36F8F704702690B46D2E948
:104C8000010183E803000020704743681B68D3F8E4
:104C90008004C3F88004704742681368D3F8580151
:104CA00040B95268920706D4D3F82001003818BFE3
:104CB0000120704701207047436802691B68D3F8E0
:104CC000100148B1527C0A700020C3F81001D3F8DB
:104CD000102101221A6070474FF0FF30704710B565
:104CE0000022044601210220FCF700FB0220FCF711
:104CF000DFFA2046BDE81040FDF798BA10B5002253
:104D0000044601212820FCF7F1FA2820FCF7D0FA0C
:104D10002046BDE81040FDF789BA704708B500206D
:104D2000FCF706FEFFF7F0BA08B5FBF753FFFCF7F8
:104D300005F8BDE80840FFF7E7BA08B50020FCF722
:104D4000C7FA18B9BDE80840FCF7B2BA08BD004779
:104D500000F0C8B9F7B5019001A8DDE9084617468B
:104D60001D46FDF74FFE019B002F00EB830014BF93
:104D700002230023002918BF43F00103002D14BFB4
:104D80004FF00C0C4FF0000C002C43EA0C0314BF46
:104D90004FF4E06C4FF0000C002E43EA0C03D0F807
:104DA000002714BF4FF4403C4FF0000C43EA0C03C3
:104DB00022EA030301B109780FB13F787F0019435C
:104DC0000DB12D78AD0039430CB1227814020D439A
:104DD0000EB1367836042C433443C0F8004703B094
:104DE000F0BD1FB50DF10F03019300238DF80F10D7
:104DF00000931A461946FFF7ADFF05B05DF804FBB6
:104E0000FEF758BA08B5FFF7FBFF002008BD704752
:104E100038B1C3681888C0F30800A0F58073584201
:104E200058417047F8B505460E464FF02003EFF3A2
:104E3000118783F31288BFF36F8FFEF7AFFF314600
:104E400004462846FFF76AFF87F31188BFF36F8F88
:104E50002046BDE8F840FCF765BC08B5FCF7B8F89B
:104E6000BDE80840FFF759BF30B50024846141EA2E
:104E7000020414F00304C0E9023201610CD1446160
:104E8000A34203D1C0E90000002030BD45690D6098
:104E9000013441611144F3E76FF01500F5E7F8B50F
:104EA00004460D464FF02003EFF3118683F312887A
:104EB000BFF36F8F476977B900F0B2F858B12A682D
:104EC0004261876700F04DF8314604F10800BDE803
:104ED000F840FEF7A7BC2B6862691A602B68636113
:104EE000A369013BA36186F31188BFF36F8FF8BDFF
:104EF00003460020C3E90200C3E900337047D0E94C
:104F0000003213605A600023C0E90033704708B5CF
:104F1000FFF7F5FF437B23F0020343730023836015
:104F200008BD034620B9EFF305820AB9FCF712BAAF
:104F300083F31188BFF36F8F70474FF02003EFF3B7
:104F4000118083F31288BFF36F8FFFF7EABF034628
:104F50000068834203D0002838BF0020704700203B
:104F6000704710B54FF02003EFF3118483F31288DC
:104F7000BFF36F8FFEF71CFD84F31188BFF36F8FB3
:104F800010BD10B501464FF02003EFF3118483F3F9
:104F90001288BFF36F8F10F80B3C13F0280F0DD160
:104FA00051F8103C18380BB1FFF7B1FF11F80B3C6A
:104FB00023F0140301F80B3CFEF7FAFC84F311888C
:104FC000BFF36F8F10BD38B504460D46FEF746FDA2
:104FD000637B43F002036373B5B12B68A5609D4208
:104FE00008BF0023002B38BF00239BB194F90E109B
:104FF00093F90E20914208D0521A002A05DD5A6812
:10500000C4E9003214605C6038BD6A68934201D024
:105010001B68EAE76B68C4E900531C606C60F3E747
:1050200038B54FF02003EFF3118583F31288BFF3F7
:105030006F8FFFF78CFF044620B1FFF768FF183031
:1050400000F00CF885F31188BFF36F8F204638BD50
:10505000EFF30580003818BF0120704710B54FF0FE
:105060002002EFF3118482F31288BFF36F8F03687D
:105070003BB1FEF7CFFF002084F31188BFF36F8FA1
:1050800010BD6FF01500F7E710B54FF02003EFF3F8
:10509000118483F31288BFF36F8FFEF7D5FF84F37B
:1050A0001188BFF36F8F10BD70B504460D464FF0E9
:1050B0002003EFF3118683F31288BFF36F8FFEF79F
:1050C000C3FF012805DDA04203DB29462046FDF78A
:1050D0005DFB86F31188BFF36F8F70BD08B5FFF7D6
:1050E000D3F808BD08B1FCF739BC70477047000021
:0450F000FDF7F8BF11
:0850F4003CB0FF7F0100000049
:1050FC00CD18000000000000111A00005C510000E7
:10510C00054E0000000000006935000000000000A2
:10511C00111E00008C510000111E00007451000083
:10512C00254D000000000000FD4C0000A4510000C3
:10513C00DF4C0000BC510000911C0000000000007E
:10514C001926000000000000294D0000000000009E
:10515C00EA550000F8530000E05300003C01002029
:10516C001C0800206C5300004C5500003854000003
:10517C0014540000440100207808002066530000FD
:10518C00F055000048540000145400004001002069
:10519C008408002060530000F75500008C54000078
:1051AC0058540000480100203C0000205A530000D5
:1051BC00FE5500006C540000585400004C010020B7
:0851CC002800002054530000EC
:1051D400112900004F4D0000000000006F4900003D
:1051E400BC510000074C0000000000006F490000A3
:1051F400000000006F490000000000006F4900003B
:10520400DD2E00004F4D0000000000006F4900003B
:10521400000000006F490000000000006F4900001A
:10522400000000006F490000000000006F4900000A
:10523400000000006F490000000000006F490000FA
:10524400000000006F490000000000006F490000EA
:10525400000000006F490000000000009D260000CF
:10526400000000006F490000000000006F490000CA
:10527400000000006F490000000000006F490000BA
:10528400000000006F490000000000006F490000AA
:10529400000000006F490000000000006F4900009A
:1052A400000000006F490000000000006F4900008A
:1052B400000000006F490000000000006F4900007A
:1052C400000000006F490000000000006F4900006A
:1052D400000000006F490000000000006F4900005A
:1052E400000000006F490000000000006F4900004A
:1052F400000000006F490000000000006F4900003A
:10530400000000006F490000000000006F49000029
:10531400A4510000074C0000000000006F49000089
:10532400000000006F490000000000006F49000009
:10533400000000006F490000000000006F490000F9
:10534400000000006F490000000000006F490000E9
:1053540000800080FF7F00800080FF7F008000804D
:0E536400FF7F00800080FF7F00800080FF7FC1
:0E537200FFFFFFFFFFFFFFFFFFFFFFFFFFFF3B
:105380000338FDD87047000000000000C947000046
:10539000750C00002D0C0000E50C0000E10B000076
:1053A0001800002000000020100000200000000075
:1053B00008000020000000200000000000000B0694
:1053C00002000000C853000000000000D555000096
:1053D0002600020700000020DD55000022000B110E
:1053E000511B0000054B00002D4B00000000000089
:1053F0003B4A000000000000C11A0000251B00000D
:10540000F34A0000F94A0000B919000071190000C0
:1054100000000000491E0000634B0000714B0000BB
:10542000874B0000934B00009F4B00003D1D000088
:10543000B14B000000000000FFFFFFFF0000005024
:105440000000000000000000FFFF0000000300500B
:105450000000000001000000B94C000029210000FC
:105460008B4C0000A51F00007B4C0000002000407A
:10547000020000000000000006000000080000001C
:10548000050000000700000001010000008002404C
:1054900002000000000000002200000021000000C7
:1054A000FFFFFFFFFFFFFFFF01000000FC500000B7
:1054B0004C510000545100005C5100005C51000050
:1054C000F5FFFFFFFF8FFFFFFF8FFFFFFE8FFFFF47
:1054D000FE8FFFFFFD8FFFFFFC8FFFFFFC8FFFFFA5
:1054E0006D757465785F667265652063616C6C6567
:1054F000642077697468204E554C4C20706172614D
:105500006D6574657200000043616E277420696EDA
:10551000697469616C697A65206D757465782C2091
:10552000776173204E554C4C0D0A0000436F756C2B
:1055300064206E6F74206C6F636B20706F77657280
:105540002073617665206D75746578004750494F0A
:105550005F3000286E696C29006D757465785F692D
:105560006E69742063616C6C65642077697468206F
:105570004E554C4C20706172616D657465720043CC
:105580006F756C64206E6F7420616C6C6F636174F6
:1055900065206D75746578206265666F7265206937
:1055A0006E697469616C697A696E67004661696CDD
:1055B000656420746F207265626F6F743A20737037
:1055C000696E6E696E6720656E646C6573736C7965
:1055D0002E2E2E0A00464C4153485F300053524154
:1055E0004D5F3000000001000000434C4F434B0072
:1055F0004750494F5F3100554152545F310055418A
:1056000052545F3000000000000001010000000063
:10561000005465726D696E616C00525454005345BC
:1056200047474552006D61696E0076322E372E393C
:10563000392D6E6373312D31002A2A2A20426F6F73
:1056400074696E67205A6570687972204F532062C2
:1056500075696C64202573202573202A2A2A0A0084
:105660005001002001000000640100200100000042
:1056700078010020010000008C01002001000000E2
:1056800027490000854900000000000000C2010019
:105690000001030000000000000000000000000006
:1056A00000C2010000010300000000000000000033
:1056B00000000000000000000000000000000000EA
:1056C00000000000000000000000000000000000DA
:1056D00000000000000000000000000000000000CA
:1056E00000000000000000000000000000000000BA
:1056F00000000000000000000000000000000000AA
:105700000000000000000000000000000000000099
:105710000000000000000000000000000000000089
:10572000FF0000000000000000000000FFFF0F006D
:105730000090D003D4000020D4000020000000001E
:1057400041430000880900201100000009440000C6
:10575000B543000025440000DD4300002001002087
:10576000E4000020180100200000000010010020CB
:105770008C09002011000000900900201100000099
:105780009409002011000000000100200C010020FD
:0C57900004010020FC000020300100207B
:10579C0000000000000000000000000000000000FD
:0457AC0000000000F9
:1057B0005001002050010020000000000000000007
:1057C0000E000000640100206401002000000000C1
:1057D000000000000E000000780100207801002089
:1057E00000000000000000000E0000008C010020FE
:1057F0008C01002000000000000000000E000000EE
:040000030000145194
:00000001FF
